:020000040000FA
:020000004F2887
:080008000B100608090003308B
:100010008800081508190A280310890D0310890D96
:1000200009088F0008000B308800081508191628E9
:100030000908900008000D100F098100051510082F
:1000400091009103031D212885151008910091034B
:10005000031D272885110108031D1F28051108000D
:100060000D1405150F088F078F070F098100100861
:1000700091009103031D3928851510089100910303
:10008000031D3F2885110108031D372805110800AD
:1000900007200F0981000108031D4B2808000301F8
:1000A0008B008A00203083000730810002308800F6
:1000B00003308500F73086008301850186018D01BC
:1000C0008B01861500001320072006089400C0301D
:1000D00094050319B128861B702830204820612818
:1000E000061B75281B2048206128861A8D280F09B9
:1000F00081000515100891009103031D7C288515CA
:10010000100891009103031D822885110108031D29
:100110007A28861E772805116128061A9928FF304B
:1001200092000A10061DDB28861CCA28061CB92866
:10013000612803018100810A0108031DAB28051114
:10014000851186118801000088308B000000630053
:1001500000008B016128F4300605F43C031D612882
:100160009C280D1CB6281B204820612830204820E0
:1001700061280A14920A120800210A1082074820F6
:1001800048204820B9281B204820B9283020482082
:10019000B92861280A14920A12081D210A10820740
:1001A000482048204820CA281B204820CA28302040
:1001B0004820CA2861280A14920A12084E210A10FF
:1001C0008207482048204820DB281B204820DB28C5
:0801D00030204820DB286128E3
:1002000082070734073404340034043407340734D5
:100210000034073404340434043404340034073420
:100220000434043404340034043407340734003410
:1002300007340434043407340A348207043407349E
:1002400004340034043404340034043404340434F6
:1002500000340734043407340434003404340734DD
:1002600000340034043404340034073407340734D1
:1002700000340734073407340434043400340434BD
:1002800007340734073407340034043407340434A3
:10029000043400340734073407340A34820707343F
:1002A0000434043404340034043407340434003493
:1002B0000434043400340434073400340734043480
:0202C0000A34FE
:00000001FF
